:020000040000FA
:020000000428D2
:08000800FF30A100FF30A2004F
:10001000962119149914191599130030A621A115C8
:10002000A5210030A021A401A501A601A701A801D6
:10003000A901AA01AB01AC014221D5202808033C4B
:10004000031DD328A508031D2628A9012508013C66
:10005000031D2C281430A9002508053C031D322857
:100060002830A9002508073C031D38283C30A9008A
:100070002508033C031D3E285030A90025080B3CF1
:10008000031D44286430A9002508093C031D4A28A3
:100090007830A90025080D3C031D50288C30A9009C
:1000A00025080C3C031D5628A030A9002508083C53
:1000B000031D5C28B430A90025080A3C031D6228F2
:1000C000C830A9002508023C031D6828DC30A900BF
:1000D0002508063C031D6E28F030A90025080E3CBB
:1000E000031D7428FF30A9002608043C031D79284D
:1000F000AA012608063C031D7F280130AA00260815
:10010000023C031D85280230AA00A608031D8A2888
:100110000330AA002608053C031D90280430AA00DD
:100120002608013C031D96280530AA002608033C3A
:10013000031D9C280630AA002608043C031DA428A1
:1001400023129E21A3129D21A608031DAB2823166E
:100150009E21A3129D212608023C031DB3282316CD
:100160009E21A3129D212608063C031DBB282316B1
:100170009E21A3129D212608053C031DC32823129E
:100180009E21A3169D212608013C031DCB28231286
:100190009E21A3169D212608033C031DD32823126C
:1001A0009E21A3169D211D28D4282521AD001430A1
:1001B0002D020318DC28D528AE010430AF0003104F
:1001C000AE0D2521B0000A3030020318E9282E10A8
:1001D000EA282E14AF0BDF282E08A500AE0103304D
:1001E000AF000310AE0D2521B0000A303002031815
:1001F000FB282E10FC282E14AF0BF1282E08A60089
:10020000AE010230AF000310AE0D2521B0000A3060
:10021000300203180D292E100E292E14AF0B0329BE
:100220002E08A700AE010230AF000310AE0D25214D
:10023000B0000A30300203181F292E1020292E1476
:10024000AF0B15292E08A8000800B1019B218519C4
:100250002A293329231129082C02031830292315B0
:100260009F21AC0A27299B21851D37293F29013071
:1002700064211E30310203183E29B10A34299B2122
:1002800031080800C830AD0023169E2101307D21C1
:1002900023129E210F306421AD0B442904305D21CF
:1002A000C830AD0023169E2101307D2123129E21EE
:1002B00014306421AD0B52290800AD002D08B300A5
:1002C0006430B4000A306B29B2003208B300013048
:1002D000B40001306B29B500FF30B6003408B80017
:1002E0003308B7001730360703187329B70B722984
:1002F000B80B7029B50B6E290800AE002E08AF00B0
:10030000AF08031D842988290A308921AF03802979
:100310000800B000F430B100FC30B2003008310702
:10032000031C003432070318922908008316FF23A8
:1003300090008312080064000800A229A229A229C3
:10034000A300A229230885000800A829A100A82944
:0603500021086500080011
:02400E0084111B
:00000001FF
